:020000040000FA
:060000006D3001303A28CA
:08000800A000030EA100831209
:1000100005191028831601178312B23081002B288E
:1000200083160113831203140B190310A80DA90DD5
:10003000AA0DAB0DAC0DAC16FF302C02031D2B2806
:10004000FA302B02031D2B2831152A08AF0029088E
:10005000AE002808AD008B100B11210E8300A00EFE
:04006000200E090065
:0C007400203084008001840A80300402E7
:10008000031C3C281230B000162283160C30850564
:1000900087018312850187010730990000309A009B
:1000A000103083168E008312603083168F00831207
:1000B0000030831691009F008312C83083168100A0
:1000C000831231309000003083168C008312103080
:1000D0008B00BC1B6D28851D89227D2281018E012C
:1000E0008F010B118B100B108C018B178520311990
:1000F0008820B30B8328031085190314B90DF03041
:10010000390203198221AE227628640032100800D9
:1001100031110130B7008B132030370783169B0055
:100120001C141A088312A4001030370783169B0092
:100130001C141A088312A300A6000230A606003081
:10014000370783169B001C141A088312A200A7000D
:100150000130A7068B17321CB32822090339A200ED
:10016000A309A409A50924082F02031D7C2923083B
:100170002E02031D192922082D02031D7C2901309E
:100180003702031DC8283D18C8283D143E143622E6
:1001900002303702031DD128BD18D128BD143E14EA
:1001A000382203303702031DDA283D19DA283D15BD
:1001B0003E143A2204303702031DE328BD19E32818
:1001C000BD153E143C2205303702031DEC283D1AB4
:1001D000EC283D163E143E2206303702031DF5285A
:1001E000BD1AF528BD163E14402207303702031D04
:1001F000FE283D1BFE283D173E14422208303702E0
:10020000031D0729BD1B0729BD173E1444220930D1
:100210003702031D10295318102953143E14472286
:100220000A303702031D1929D3181929D3143E1493
:10023000492226082E02031D7C2927082D02031DB2
:100240007C2901303702031D2A293D1C2A293D1033
:100250003E144B2202303702031D3329BD1C3329C3
:10026000BD103E144C2203303702031D3C293D1DB6
:100270003C293D113E144D2204303702031D45290F
:10028000BD1D4529BD113E144E2205303702031D08
:100290004E293D1E4E293D123E144F220630370294
:1002A000031D5729BD1E5729BD123E145022073089
:1002B0003702031D60293D1F60293D133E14512262
:1002C00008303702031D6929BD1F6929BD133E147B
:1002D000522209303702031D7229531C7229531010
:1002E0003E1453220A303702031D7B29D31C7B297D
:1002F000D3103E1455227C29B70A0B30370203185D
:1003000008008B280130B600B300B400B500B70078
:1003100085018701B1138520B30BC229031085190C
:100320000314B90DF03039020319E929B40BC229BD
:100330000130370203195F220230370203196222AB
:10034000033037020319652204303702031968228B
:100350000530370203196B220630370203196E226B
:10036000073037020319712208303702031974224B
:1003700009303702031977220A30370203197A222B
:100380009630B400311D8B293111321CCC292D0936
:100390000339AD00AE09AF092F1C8B298E018F01E7
:1003A0000C1C8B290C102E1E8B298B132030370729
:1003B000BB002F08BA00012210303707BB002E08FF
:1003C000BA00012200303707BB002D08BA00012215
:1003D0008B1785018701B70AB6010B303702031C62
:1003E0008B297D2208003E1C08003E101030BB0007
:1003F0003D08BA0001223030BB005308BA00012288
:1004000008008B133A0883161C159A0083123B08C8
:1004100083169B0055309D00AA309D009C146400FB
:100420009C180F2A1C1183128B17080083160030AA
:100430009B001C141A088312BC00831610309B000A
:100440001C141A088312BD00831630309B001C1444
:100450001A088312D300FF30D000D415D515D61555
:10046000D715D915DA15DB15DC150800F130572A38
:10047000F230572AF430572AF830572A1F305B2AB7
:100480002F305B2A4F305B2A8F305B2A080087149D
:100490000800071508000800080008000800080008
:1004A0000800080008008710080007110800BD05B3
:1004B0000F30D2040800BD05F030D204080010301F
:1004C00085060800203085060800213085060800D2
:1004D000223085060800183087060800213087067C
:1004E0000800093087060800293087060800023016
:1004F0008706080004308706080053188714D318AD
:1005000007153D08D200031D08001130BD00D200C0
:100510000800B601B301B4013C1C912ABC01BC1413
:10052000932ABC013C143C08B6006400972A982A20
:10053000992A9A2A9B2AB41B0516B41F0512B30BDD
:10054000952AB40B952A0310B60CB608031D952AFC
:100550000030BB003C08BA00012208008F080319D4
:1005600008008F01D00FC82BD00A0E305205031D92
:10057000C82A541DBE2AD4015416D62AD41DC32A13
:10058000D4015416D62A541ED62AD401D414D62AFD
:10059000D41CCD2AD4015415D62A541DD22AD401F4
:1005A000D415D62A541ED62AD4015415013052052A
:1005B000031DE92A551DDF2AD5015516F72AD51D39
:1005C000E42AD5015516F72A551EF72AD501D51468
:1005D000F72AD51CEE2AD5015515F72A551DF32A01
:1005E000D501D515F72A551EF72AD50155150B301B
:1005F0005205031D0A2B561D002BD6015616182B2B
:10060000D61D052BD6015616182B561E182BD601B3
:10061000D614182BD61C0F2BD6015615182B561D89
:10062000142BD601D615182B561E182BD60156158D
:1006300007305205031D2B2B571D212BD7015716B1
:10064000392BD71D262BD7015716392B571E392B7F
:10065000D701D714392BD71C302BD7015715392B7D
:10066000571D352BD701D715392B571E392BD701DD
:1006700057151030BC1811305205031D4E2B591D53
:10068000442BD90159165C2BD91D492BD901591678
:100690005C2B591E5C2BD901D9145C2BD91C532B14
:1006A000D90159155C2B591D582BD901D9155C2B33
:1006B000591E5C2BD90159155030BC1851305205C8
:1006C000031D712B5A1D672BDA015A167F2BDA1D79
:1006D0006C2BDA015A167F2B5A1E7F2BDA01DA14A3
:1006E0007F2BDA1C762BDA015A157F2B5A1D7B2BB8
:1006F000DA01DA157F2B5A1E7F2BDA015A15E0300A
:10070000BC18E1305205031D942B5B1D8A2BDB01C5
:100710005B16A22BDB1D8F2BDB015B16A22B5B1E56
:10072000A22BDB01DB14A22BDB1C992BDB015B155D
:10073000A22B5B1D9E2BDB01DB15A22B5B1EA22BCC
:10074000DB015B152030BC1821305205031DB72B8F
:100750005C1DAD2BDC015C16C52BDC1DB22BDC0156
:100760005C16C52B5C1EC52BDC01DC14C52BDC1C08
:10077000BC2BDC015C15C52B5C1DC12BDC01DC1521
:10078000C52B5C1EC52BDC015C15F3213D08D20096
:100790005008D1000C305405031D05120C305505CE
:1007A000031D85120C305605031D05100C3057052E
:1007B000031D85100C305905031D07100C305A0518
:1007C000031D87120C305B05031D07120C305C05FE
:1007D000031D871151080E020318122C1230540504
:1007E000031D051612305505031D851612305605DA
:1007F000031D051412305705031D851412305905C9
:10080000031D071412305A05031D871612305B05AD
:10081000031D071612305C05031D8715FF305002BB
:10082000031908008F08031D0800852051080E02D7
:10083000031C122C18305405031D051206305405F4
:10084000031D051618305505031D85120630550584
:10085000031D851618305605031D05100630560574
:10086000031D051418305705031D85100630570564
:10087000031D851418305905031D0710063059054E
:10088000031D071418305A05031D871206305A0538
:10089000031D871618305B05031D071206305B0524
:1008A000031D071618305C05031D871106305C0513
:0608B000031D871508007E
:084000000400030005000900A3
:02400E00CC33B1
:10420000010078007A007C007E007B0079007F004E
:104210007D007A0078007E007C00FF00FF00FF0038
:104220000000F200F600FA00FE00F200F600FA00CC
:10423000FE00F200F600FA00FE00FF00FF00FF00A3
:10424000010005000500050005000900090009003E
:1042500009000D000D000D000D00FF00FF00FF0024
:10426000FF00FF00FF00FF00FF00FF00FF00FF0056
:10427000FF00FF00FF00FF00FF00FF00FF00FF0046
:10428000FF00FF00FF00FF00FF00FF00FF00FF0036
:10429000FF00FF00FF00FF00FF00FF00FF00FF0026
:1042A000FF00FF00FF00FF00FF00FF00FF00FF0016
:1042B000FF00FF00FF00FF00FF00FF00FF00FF0006
:1042C000FF00FF00FF00FF00FF00FF00FF00FF00F6
:1042D000FF00FF00FF00FF00FF00FF00FF00FF00E6
:1042E000FF00FF00FF00FF00FF00FF00FF00FF00D6
:1042F000FF00FF00FF00FF00FF00FF00FF00DD00E8
:00000001FF
